:020000020000FC
:0E0000000EC00DC00CC00BC00AC009C008C065
:10001C0028C0A8950FE50DBF08E00EBF00270ABB4E
:10002C000FEF0BBB09EF09BB002707BB00EF08BBA9
:10003C000FEF04BB002705BB002702BB0FEF01BB72
:10004C0091D35BD2BBD368D24FE0F8D23FE0DAD188
:10005C00AA24BB24CC248824992478940000000082
:10006C00FDCF8395843108F08827B5D357D11FE78E
:10007C00111611F4949801C06CD07BD0F22E60FF55
:10008C001895022F0670003009F411D0023009F4D3
:10009C0016D0043009F41FD0063009F434D0D0D077
:1000AC00882321F4B4D025D2B6D1ACD1189563FFF6
:1000BC00089534D11FE7111609F032D00895092C98
:1000CC0011245ED109E1112772D1902C63FF0895A0
:1000DC00092D26D008950EE30623A1F06068F0E008
:1000EC00E0E6092D000FE00F019000810F77102E34
:1000FC0047D107EE13E05BD11082029263FF0895A3
:10010C00092D0ED00895AA240B2C1C2C0F2D07FFA3
:10011C0058D136D113E007EE4AD1B02CC12C08953A
:10012C00F0E0E0E6000FE00FE395008110E8012716
:10013C0000830895949B089563FF08959498F0E0CC
:10014C00E0E6092D000F0395E00F008100680083A5
:10015C000895F0E0E0E6000FE00F019010811F77AA
:10016C00112E0B181C081CF011F094980895949AF9
:10017C00089529B3022F06701F2D1670012719F050
:10018C0088246078089583940FE7801608F0802EF9
:10019C0060FD0DC00AE080160CF40895616088249F
:1001AC00022F0670043019F067FDEBD26F7725FF34
:1001BC000BC06F7E6D7F24FF13C06F7D6B7F27FF9D
:1001CC001BC0677F88240895F5FE03C062608824F5
:1001DC0008956D7F0EE180160CF40895606108950A
:1001EC00F4FE03C06460882408956B7F0EE18016D2
:1001FC000CF4089560620895F7FE03C068608824CB
:10020C000895677F0EE180160CF4089508950F2D64
:10021C0006700630A1F009B303FF11C001E0A00E77
:10022C000CE3A01664F0AA2401E0B00E0027C01E57
:10023C000B2C1C2C07EE13E0BAD0B02CC12C08955B
:10024C005FD010E28AD11F2D1670103069F0163075
:10025C0059F003E582D105E4123021F07ED104E59A
:10026C007CD127C00CE425C004E577D176D107E416
:10027C0074D100E472D152D0112D1F3741F4F7E044
:10028C00ECEE9FD10F2D0670063081F008950F9380
:10029C0011E6010F62D10F9157D055E0E6E0FF2730
:1002AC008AD10F2D0670063009F0089502E85AD154
:1002BC00089500E452D101E6090D4FD1F0E0E0E6DB
:1002CC00092D000FE00F0190008107FB0F77102E16
:1002DC007ED196D18BD001E2602E16F40FE3602E06
:1002EC0055E0E6E0FF2767D10F2D0670023011F0C4
:1002FC00043019F00BE836D108950FE833D1089586
:10030C0000E830D161D053E0E6E0FF2754D10AE396
:10031C0024D152E0E3E0FF274ED108950FE7102ED1
:10032C00F0E0E0E6E43978F4219111911123D2F355
:10033C0011151CF0B9F70216A8F3112E022E0E2F70
:10034C0002560695EFCF0895F0E0E0E6000FE00FBF
:10035C00019010811F77112E0B181C0824F037D137
:10036C004FD144D008950094109401E0000E002762
:10037C00101E2DD145D13AD00DE2E395008308959E
:10038C0061FD09C064FD05C062FD0CC065FD08C0BF
:10039C00089580FF089501E0000E0027101E0895B7
:1003AC0080FF089501E0001A0027100A0895111625
:1003BC0034F009F002C0001614F0112E002E11209A
:1003CC0014F41124002408950B2C1C2C00D118D1EA
:1003DC000DD05F924F923F922F920A2C1124F7D09E
:1003EC000FD14F905F906F907F90089525E0E7E0DC
:1003FC00FF271081103329F410E21083EA952A9517
:10040C00C1F7089541E04DD142E04BD144E049D1D0
:10041C0048E047D108950DE0DAD10AE0D8D1606404
:10042C0041E0432311F497D102C041D123D042E0E3
:10043C00432311F490D102C03AD11CD044E04323A1
:10044C0011F489D102C033D115D048E0432319F4FB
:10045C0082D16F7B08952BD10DD06F7B089501E075
:10046C0081D002E4302E0DE3202E52E0E3E0FF2792
:10047C00A2D0089517FA17FE04C0019400E00109F8
:10048C00102E102D1F7024E0159407942A95E1F777
:10049C0013FF03C003940BF413940F2D06FD0ED021
:1004AC0096D0AED0A3DF1EF4E3951DE2108353E08B
:1004BC00E4E0FF2780D000E250D0089519E0019EBF
:1004CC00002D112D1124A5E0BB2732D11D2D133089
:1004DC0008F0039510E22EF0010F48F40FEF002EF8
:1004EC000895E894101B012F10F401956894002EC8
:1004FC00089500EC45D036D008951FD00CE332D0CF
:10050C0031D030D02FD006E02DD00EE02BD001E032
:10051C0029D000E827D0089500270EBD0FBD0DBDD2
:10052C000CBD02E00BBD0BEB0ABD882700E109BF37
:10053C000CE00EBD00270FBD0895002703BF02BFBE
:10054C0009BF01E008BF05E003BF01EF02BF08B718
:10055C0000FFFDCF002703BF089566FD38D1959AA3
:10056C00969803C09598969800C00AD005BB0000D9
:10057C000000979A0000000000009798AF9808952B
:10058C000F9302B30F93002704BB9598969A000023
:10059C0000009798000000000000979A00000000EF
:1005AC0000009F99F4CF000097980FEF04BB0F91B8
:1005BC0002BB0F91089500813197CFDF5A95D9F77F
:1005CC00089555910591C9DF5A95E1F7089520E1F9
:1005DC00442433242224FF27000C111C221C331C1E
:1005EC00441C2A9509F40895E5E002910D5F03FD82
:1005FC0000830081005D07FD0083E230B1F7ECCF92
:10060C00042D0F70602E042D007F0295702E032D8B
:10061C000F70402E032D007F0295502E022D0F934C
:10062C000F70202E0F91007F0295302EE2E0FF27F5
:10063C00008100630193E830D8F308950CD07CEC72
:10064C0043D07EE441D070E03FD070E03DD07FE7F6
:10065C003BD001D00895042F00953023042F07BB05
:10066C000BEC11D000E007BB04EE0AD006B30095EA
:10067C000423302B03ED07D0089504BD01E006C020
:10068C0004BD02E003C004BD03E000C012E010BFD3
:10069C0010E418BF05BD08B706FFFDCF002705BD48
:1006AC000895D9DF7CEC10D074E40ED008952ED0D0
:1006BC00F1F3D1DF7CEC08D07EEB06D01ED0072EF8
:1006CC001CD0172EC8DF089528E007B3042B07BBF6
:1006DC0070FD08C007EED4DF07B3007F07BB02EF45
:1006EC00CCDF07C009EFC9DF07B3007F07BB07EEFC
:1006FC00C7DF76952A9549F70895772728E07695F0
:10070C0005D009F070682A95D1F7089507B3042B2A
:10071C0007BB09EFB2DF07B3007F07BB0DEFADDFFF
:10072C0016B314231F930BEEABDF1F911123089507
:10073C00DD24EE18B1E1001F111FBA9509F40895DC
:10074C00DD1CEE1CDA1AE20A20F4DA0EE21E8894A2
:10075C00F2CF0894F0CFEAE6F7E033DF08950453C4
:10076C00656E200010E01FBBE0E6F0E010E0E199C0
:10077C00FECF1EBBE09A2DB321931395E439B8F349
:10078C0008952F9310E01FBBF0E0E0E6092D000F59
:10079C00E00F10E0092D000F100FE199FECF219111
:1007AC001EBB2DBBE29AE19A1395E199FECF2191E4
:1007BC001EBB2DBBE29AE19A2F91089510E006E141
:1007CC0010BD09B908E10AB90EE800BD08955D9B9A
:1007DC00FECF0CB908955F9B08950CB1F8DF089516
:0807EC0006204E6F416374000A
:00000001FF
